:030000000200807B
:030003000202FDF9
:03000B00020210DE
:0300130002015E89
:03002300020BB11C
:03002B0002022BA3
:03005300020D3962
:100080007590FE75B0DFC291C2B47581AF75D010A6
:100090001201A175D700759C0075892275870075BE
:1000A000987075CBFF75CAC975C83475880075EF2F
:1000B0009075D80075F50075FD9F75A80075243002
:1000C0001202CC120248901C661208EF901C7712A4
:1000D00002841208EF901C881202881208EF790936
:1000E0007C001202C5D9F9901D601209241207196B
:1000F00012010EA20F921785323485333512045740
:100100001208F47581AF1201A175A89580F5E4F588
:1001100022F520F521120AE9120B38120B611207A1
:100120005BC204C2901201C4120626E4F5A1F5A335
:10013000F5A4F5A575A64075A10375A904E5306081
:1001400018B42B005013D208C32323F58275831AE9
:10015000E493F529A3E493F52AC299C29822C2AA8E
:10016000C2AFC0D0C0E0C0F0C082C08375D000D2A2
:10017000B4C2251202CC120656300803120634C24D
:10018000AA1201A1D2AF30B3FD1202C330B3F7C23D
:10019000AF31B1D083D082D0F0D0E0D0D0D2AAD2CB
:1001A000AF32901CEE300E03901CDD12028002086C
:1001B000EFD2251202CCC290C2B53008031206114C
:1001C000C2B4C2041201D331A28533358532341250
:1001D000045722855837855938855A39855B3A0244
:1001E00007B620090F855137855238855339855414
:1001F0003A0207B6C3E5549562F53AE5539561F5C1
:1002000039E5529560F538E551955FF5370207B647
:10021000C0D0C0E0E8C0E0A82E86F908B890027807
:1002200080882ED0E0F8D0E0D0D032C0D0C0E0E856
:10023000C0E0C2CFA82F86FB08B890027880882F34
:10024000D0E0F8D0E0D0D032C220C2211202CC746B
:10025000391202A474151202A474551202A4746E09
:100260001202A474721202A474381202A4740C1242
:1002700002A474011202A47C021202C57406802436
:10028000748080067490800274A0C2201202CC8018
:1002900013E53B519FE53C519FE53D80027420D220
:1002A000201202CCC0E07472120897D0E01208A8A5
:1002B000120857D2221202CCC2221202CC227F2074
:1002C000DFFE227C13E41470FDDCFA22C0E07474BB
:1002D000120897E5241208A8D0E0020857E4752216
:1002E0000002010374791208971208BFF52B51C35D
:1002F00074791208971208BFB52BE6F422C2AF51E9
:10030000E460DE20B3030203D730E007C2E070CD23
:100310000204CB30E307C2E370C30205AA30E11D3B
:10032000C2E170B9B21130110F901D10518812083E
:10033000EFE53612057D80A912044B80A430E2233C
:10034000C2E270990525E525B40600400375250035
:10035000120A2B120AE912043231B131A21208F446
:100360000202E130E423C2E47010B21230120E90A7
:100370001D4C51881208EF0205130202DD1209F725
:10038000120A091208F40202E130E64BC2E670EAF2
:10039000B216301603020475E5317006C20BC209AD
:1003A000802CB40107D20B1204328022B40204D292
:1003B0000E8005B40309C20E120B4B31A2800FB49C
:1003C0000406D20CD2248004C20CC22451CC120ADE
:1003D000091208F40202E130E53EC2E5709CD291B8
:1003E000C2A830B312D2B4C22551CC12065675A899
:0E03F0000030080312063431A11205F2D2AF1C
:1003FE0020B2FD51E420E5F8C29112060930B30790
:10040E00C2AF31B1020103D2A832C2E77013B217E4
:10041E00A217920F120A091208F420B304A217921F
:10042E00B50202E1C209300B13E533B4020EE53218
:10043E00B4A9005007B46C004002D20922120B740A
:10044E001209E51208F41209805184901D21300919
:10045E0003901D321208EF7493518AA934A83512F5
:10046E0006B10202910531E531B406004003E4F510
:10047E0031901C55B40005901C008020B4010590ED
:10048E001C118018B40205901C228010B403059034
:10049E001C338008B40405901C4480005188120857
:1004AE00EF0202E1E536B401057536058006B405A6
:1004BE000375360A12057D120B740202E12011E457
:1004CE0020123920169FE533B40210E532B4BC0B6E
:1004DE00753300753200120A6C800FE5362532C571
:1004EE0032E5333400C533120A3B120980913231A2
:1004FE00D385323485333591570202E1E530B42A83
:10050E000280020530E530700F901D4374A7518AAA
:10051E001208EFC2080202E1D208C32323F5827546
:10052E00831AE493F529A3E493F52AA3E493120620
:10053E00EEF543E5F0F542B53003754220A3E493A2
:10054E001206EEF54675452EE5F0F5447547207515
:10055E00484875497A74A7518A7842E6519F08B87F
:10056E004AF90202E1E5307002809A1530809674E5
:10057E00A4518AE536753B20B40108753C20753DC3
:10058E00318011B40508753C20753D358006753CEB
:10059E0031753D30020291153102047520112D2066
:1005AE0012C32016F2E5337010E532700C7533026B
:1005BE007532BC120AC40204F8E532C39536F53220
:1005CE00E5339400F533120A910204F8E536B40AC5
:1005DE00057536058006B40503753601B17D120B1F
:1005EE00740202E1758ACE758CCE43FD03752E80A2
:1005FE0075F99F75FB9FD28CD2A922C28CC2A953CA
:10060E00FDFE22C2CAC2AD53FDFD75CBFF75CAC930
:10061E0075C834C299C29822901B007880E493F674
:10062E00A308B890F822C2CA75C8008529CB852ABE
:10063E00CA8529CD852ACC43FD0375F99F75FB9F8D
:10064E00752F80D2CAD2AD2285333585323430092A
:10065E0007E532C39464C534D20431E2A21792B5D1
:10066E00D290901CFF51801208EF91572278547946
:10067E00578004785B795E7B03C3E736C61819DBB7
:10068E00F95004E63400C622785479578004785B1A
:10069E00795E7B03C3E697C61819DBF950E9E69439
:1006AE0000C622E4FAFBFC7D10E933F9E833F8ECDE
:1006BE003CD4FCEB3BD4FBEA3AFADDEDEB540F44B1
:1006CE0030F53BECC4540F4430F53CEC540F443041
:1006DE00F53D221206EEC5F0120930C5F0020930C2
:1006EE00C0E0C41206F8F5F0D0E0540FB40A004092
:1006FE00022407243022B43A0040029407540F22F9
:10070E0075C60075B901E5BC60002275C60B75B9DA
:10071E000185BC2585BF4F1208951208573000126F
:10072E00901D5DE493601FF54F1208951208572037
:10073E000011901B5C120924E54FD1E11209291218
:10074E000A1B22A380DD901B4312092422755087B9
:10075E00120895E5501208A874011208A81208573D
:0E076E000202C3755089120895E5501208A8C2
:10077C0074101208A812085722755089120895E5B2
:10078C00501208A874001208A81208572275F040DD
:10079C0020040375F050755087120895E550120827
:1007AC00A8E5F01208A812085722F1711207F8F107
:1007BC0085F199221207C71207D22275F030300446
:1007CC00D575F02080D075F0503004CA75F040809B
:1007DC00C5F17112089574071208A87B067866E6B5
:1007EC001208A808DBF9120857F185227B04755012
:1007FC0007120895200062E5501208A8200417740F
:10080C00E21208A874C21208A87837E61208A808E1
:10081C00DBF91208572274E31208A874C280E7753A
:10082C00500712084C78427B06E54FD2E01208972D
:10083C00BB01051208BFF6221208D7F6081B80F080
:10084C00120895200013E5501208A8C2B712085FD1
:10085C00D2B722D2B630B6FD22901B32C0E011576F
:10086C00D2001202881208EFD0E01206EEC0E0743B
:10087C00AE12028AE5F012029FD0E012029F229083
:10088C001B1080D8901B2180D3E54FC200D2B6D26A
:10089C00B730B6EB30B7EDC2B700C2B67F083392B3
:1008AC00B7115FC2B6DFF7D2B7115F30B702D20013
:1008BC00C2B6227F08115F00A2B733C2B600DFF5C3
:1008CC00D2B7115F00C2B6D2B780807F08115FA289
:1008DC00B733C2B6DFF7C2B7115FC2B6D2B72212B6
:1008EC00029FA3E49370F82212028830080B901C2C
:1008FC00CC300F0E901CBB8009901C99300F0390CC
:10090C001CAA11EF74A312028A7441252502029FBE
:10091C00F5993099FDC299A3E49370F422740D12E9
:10092C000930740AF5993099FDC29922742080F42B
:10093C00743D80F0786512095430011BF608B87BC1
:10094C00005014B40DF0182279027A007B00209824
:10095C0009DBFBDAF7D9F3C20122E599C298D2017F
:10096C00228566C675B90185BC6785BD6885BE697B
:10097C0085BF6A221209DB85F0C675B9018521BCD9
:10098C0075B90575B90205F085F0C675B9018533E1
:10099C00BC8532BD75B90575B90205F085F0C67513
:1009AC00B9018558BC8559BD855ABE855BBF75B9E3
:1009BC000575B90205F085F0C675B9018551BC8580
:1009CC0052BD8553BE8554BF75B90575B90222E574
:1009DC00252323232420F5F02231DB85F0C675B9BD
:1009EC00018536BD75B90575B9022231DB85F0C6B6
:1009FC0075B9018530BE75B90575B9022231DB8533
:100A0C00F0C675B9018521BC75B90575B902227599
:100A1C00C60B75B901854FBF75B90575B90222753D
:100A2C00C60B75B9018525BC75B90575B90222C30C
:100A3C00E55B355EF55BE55A355DF55AE559355C98
:100A4C00F559E43558F558C3E5543557F554E55385
:100A5C003556F553E5523555F552E43551F55122DD
:100A6C0075C61A75B90185BC5885BD5985BE5A85A0
:100A7C00BF5B75C61C75B90185BC5185BD5285BE61
:100A8C005385BF5422C3E55B955EF55BE55A955DD6
:100A9C00F55AE559955CF559E5589400F558C3E5B8
:100AAC00549557F554E5539556F553E5529555F530
:100ABC0052E5519400F5512275C61B75B90185BCE0
:100ACC005885BD5985BE5A85BF5B75C61D75B90164
:100ADC0085BC5185BD5285BE5385BF542231DB8503
:0E0AEC00F0C675B90185BC2185BD3685BE30CA
:100AFA00A20C92241202CC05F085F0C675B90185C4
:100B0A00BC3385BD3205F085F0C675B90185BC5880
:100B1A0085BD5985BE5A85BF5B05F085F0C675B996
:100B2A000185BC5185BD5285BE5385BF542275C609
:100B3A001975B90185BC5F85BD6085BE6185BF62D7
:100B4A002275C60A200E0375C60975B90185BC2C23
:100B5A0085BD2D85BE4C2231DB85F0C675B9018570
:100B6A00BC2185BD3685BE30714BE536B40A0875A1
:100B7A00C61375F0168011B4050875C61475F017FA
:100B8A00800675C61575F01875B90185BD5C85BEF8
:100B9A005D85BF5E85F0C675B90185BD5585BE56B2
:100BAA0085BF5722C299323098FAE599C298C2E5B0
:100BBA00B443F1313031403001EAE565B45FE5E52F
:100BCA0066B44112112B7B067842E61206E13138EF
:100BDA0008DBF7312932B4420A120CC61207DD12B9
:100BEA00079F32B4430D120CC61207DD75F040128E
:100BFA0007A232B4440612075B71CE32B4521B31DB
:100C0A003C756600316D7867E6081206E1B86BF844
:100C1A00056674A0B566ED312932B4573479667821
:100C2A0067E6120704C4F708E612070447F709083B
:100C3A00B96BEE8566C68567BC8568BD8569BE8564
:100C4A006ABF75B90575B902313C79143140020B96
:100C5A00B8B45367C2AF901B773124C2983098FD5D
:100C6A00E599C298B40D54120D63854A26854B271F
:100C7A00901BA73124C2983098FDE599C298B40D0B
:100C8A003A120D63120CDD75C60A854ABC854BBD46
:100C9A00854CBE75BF0075B90575B902120CF6759B
:100CAA00C609854ABC854BBD854CBE75BF0075B962
:100CBA000575B902901BD73124D2AF3279667867AD
:100CCA00E6120704C4F708E612070447F70908B84A
:100CDA0073EE22E527C3954BFBE526954AFA740580
:100CEA00120D20BB0500B33400F54C22E527C3954D
:100CFA004BFBE526954AFA741E120D20BB0F00B372
:100D0A003400F54CC333C333C54BC3954BF54BE5A0
:100D1A004A9400F54A22F42401CA7C0950042AD3D1
:100D2A0080042A40019ACB33CB33DCF013CB22C0A8
:100D3A00D0C0E0C0F0C083C08275D0081201A120E3
:100D4A00B406120D63120D97120E2575A103D082F7
:100D5A00D083D0F0D0E0D0D02275EFBC75D8027421
:100D6A00201470FDC0E0D2DC20DCFD85D94B85DA89
:100D7A004A534A0FC3E54A13F54AE54B13F54BC3E9
:100D8A00E54A13F54AE54B13F54BD0E022C202C3FC
:100D9A00E54B952DFBE54A952CFA500DD202E52D2F
:100DAA00C3954BFBE52C954AFAE54CB120FC300E75
:100DBA0038C2052002132404F5F07409B5F0009234
:100DCA0005E5F0500B74098007C374049C5001E4D4
:100DDA004430F53D748312028AE53D12029F742065
:100DEA00300502742B12029F22753B2B30020375C9
:100DFA003B2D753C00753D007D08C3EC33FC793C06
:100E0A00E737D4F7DDF409540F4430F719E7C4542F
:100E1A000F4430F71202801202912275D80374200F
:100E2A001470FDD2DC20DCFD85D94E85DA4D534D98
:100E3A000FE54DC4F54DE54E540FF5F0E54E54F06F
:100E4A00C4454DC5F0B40800B3C5F03400FD75F0D3
:100E5A006484F53BC5F075F00A84F53C85F03E43A1
:0E0E6A003E30753D2E433C30433B30748A12BF
:0B0E7800028A120291E53E12029F2246
:101A0400FAE80670FB130693FB410719FB6A0744C7
:101A1400FB910770FBB80797FBDD0825FC01085410
:101A2400FC250885FC450915FC660948FC7F0974FA
:101A3400FC961000FCB41035FCD11072FC76110930
:101A4400FD071148FD201188FD3A1230FD52127332
:101A5400FD691318FD801365FD961413FDAA146225
:101A6400FDBF1514FDD21567FDE51622FDF81669B4
:101A7400FE091738FE1A1799FE2B1862FE3B1998B7
:101A8400FE532035FE592065FE612107FE6F21813A
:101A9400FE702257FE832291FE8A2336FE97241875
:081AA400FEA32503FEA8254165
:101B00009FBFDFEFFFEFDFBF9F7F5F4F3F4F5F7FE5
:101B10004932432053434C204572726F722020207B
:101B20000049324320534441204572726F72202095
:101B300020004932432041434B206572726F72206E
:101B40002020005349353731206E6F7420666F7541
:101B50006E64206F6E204932430D0A0053493537B9
:101B60003120666F756E64206F6E204932432061AC
:101B7000646472203A2000536574207369676E6153
:101B80006C2067656E657261746F7220746F2035AA
:101B90003075562020282D373364426D29202020AF
:101BA000285339290D0A00536574207369676E61E3
:101BB0006C2067656E657261746F7220746F20317E
:101BC0002E36755620282D3130332064426D292061
:101BD000285334290D0A00525353492043616C693C
:0A1BE000627261746564200D0A0052
:101C000053494D504C4558204D4F444520202020ED
:101C1000004155544F20524550204D4F44452020FF
:101C2000200052535349204D4F444520532020203B
:101C300020200052535349204D4F444520206442F8
:101C4000755620004241434B4C49474854204F4E63
:101C500020202020004241434B4C49474854204F0C
:101C60004646202020002A2A2A2A204F5A34485A41
:101C7000202A2A2A2A2000202032394D487A205250
:101C8000582F5458202020002076657220312E30A5
:101C900020203137303332320056464F202020206A
:101CA0002020202054582048690056464F202020EC
:101CB00020202020205458204C6F0056464F2020D2
:101CC0004354435353205458204C6F0056464F20E2
:101CD0002043544353532054582048690020532034
:101CE00020204261747420202020202056002020D3
:101CF00020206442755620202020202020560020DD
:101D00005458206F6E2020202020202020205600B4
:101D100053544550202020204B487A20202020205A
:101D20000032392E202020204D487A20202053498F
:101D30004D0032392E202020204D487A20202D526F
:101D400045500064697361626C6564004354435399
:101D500053202020202020202020202000BEAA0068
:101D60004F5A34485A203239204D487A2052582F41
:101D700054582076312E3020202032303137203018
:071D8000332032320D0A008E
:00000001FF
